:020000040000FA
:100000000C94F2040C941A050C941A050C941A051D
:100010000C941A050C941A050C941A050C941A05E4
:100020000C941A050C941A050C941A050C941A05D4
:100030000C941A050C941A050C941A050C941A05C4
:100040000C941B1E0C941A050C948B1E0C94651EAC
:100050000C941A050C941A050C941A050C941A05A4
:100060000C94BD1E0C941A0500407A10F35A00A09F
:10007000724E18090010A5D4E80000E87648170071
:1000800000E40B54020000CA9A3B000000E1F505B1
:10009000000080969800000040420F000000A086FB
:1000A00001000000102700000000E803000000002D
:1000B0006400000000000A000000000001000000D1
:1000C00000002C76D888DC674F0823DFC1DFAE59EB
:1000D000E1B1B796E5E3E453C63AE651997696E87E
:1000E000E6C28426EB898C9B62ED407C6FFCEFBC02
:1000F0009C9F40F2BAA56FA5F490055A2AF75C932D
:100100006B6CF9676DC11BFCE0E40D47FEF520E662
:10011000B500D0ED902E0300943577050080841E45
:10012000080000204E0A000000C80C333333330FA0
:10013000986E12831141EF8D2114893BE65516CF3D
:10014000FEE6DB18D1844B381BF77C1D901DA4BB49
:10015000E424203284725E228100C9F124ECA1E5FE
:100160003D270000000000000000050000000A001C
:1001700000000F00000014000000190000001E0025
:10018000000023000000280000002D0000003200C5
:100190000000370000003C00000041000000460065
:1001A00000004B00000050000000550000005A0005
:1001B00000005F00000064000000ECFFFFFF274824
:1001C0000E00D7571200319D1600F5191B00EBCF1A
:1001D0001F00DEC02400A1EE29000D5B2F000208E5
:1001E000350063F73A00202B410028A547007567CA
:1001F0004E0006745500DCCC5C0005746400926B04
:100200006C0098B5740036547D008F498600CA97FB
:100210008F00F1FFFFFF87C80A0067C40E00ECF4EF
:100220001200CC5B1700C6FA1B009FD320001FE80A
:100230002500163A2B005ACB3000C89D360044B337
:100240003C00B40D430008AF49003599500035CE4D
:10025000570009505F00B72067004F426F00E0B6BB
:100260007700858080005CA18900F6FFFFFFDC3B02
:100270000700EB230B009B3F0F009790130097188C
:10028000180054D91C0091D42100130C2700A88118
:100290002C00223732005C2E380034693E008FE992
:1002A000440059B14B0082C25200011F5A00D2C80B
:1002B0006100FAC169007E0C720070AA7A00E29DAA
:1002C0008300FBFFFFFF46A30300857707005F7EE7
:1002D0000B0077B90F007D2A14001FD3180018B542
:1002E0001D0025D222000A2C280091C42D00899DD2
:1002F0003300CAB839002C18400092BD4600E4AA69
:100300004D000DE2540001655C00BA3564003356BF
:100310006C0070C874007D8E7D000000000000003D
:10032000000070C0030073B20700A9D70B00B23100
:1003300010003BC21400EF8A1900878D1E00BDCB50
:1003400023005047290008022F00AFFD3400193C5C
:100350003B001CBF4100968848006B9A4F0082F614
:100360005600C99E5E0036956600C0DB6E0068745C
:100370007700050000006053FCFF00000000EB6206
:1003800000007FEC07008E2F0C00FCA710006E57BA
:100390001500903F1A0016621F00B5C024002B5DA7
:1003A0002A003A393000AB5636004BB73C00EF5CC0
:1003B00043006F494A00A87E510080FE5800E0CA01
:1003C0006000B8E56800FA5071000A000000D89E8D
:1003D000F8FFA737FCFF000000006DF9030082253D
:1003E0000800D4850C00031C1100B1E9150086F04B
:1003F0001A003232200066B02500DD6C2B005669F1
:10040000310093A737005F293E0089F04400E5FEE4
:100410004B004E565300A2F85A00C5E76200A325D0
:100420006B000F000000F3E3F4FFF468F8FF771CA3
:10043000FCFF0000000019150400515D08003DDAC2
:100440000C00768D11009C781600529D1B0046FD15
:100450002000249A2600A4752C007F91320073EFAF
:10046000380049913F00C7784600C0A74D000720DB
:10047000550078E35C00F0F36400140000005F2492
:10048000F1FF9095F4FF3C34F8FFE201FCFF00001F
:1004900000001E300400C5930800892C0D00FFFBEE
:1004A0001100C303170075451C00BBC22100427D2B
:1004B0002700B9762D00D7B03300572D3A00F9ED5B
:1004C000400081F44700BD424F007ADA56008DBDEE
:1004D0005E0019000000E061EDFF41BFF0FF194927
:1004E000F4FFDA00F8FFFDE7FBFF00000000654ABB
:1004F0000400B4C808007A7C0D0049671200BA8A6B
:10050000170068E81C00F68122000B592800526F82
:100510002E007CC6340040603B005A3E4200886298
:10052000490092CE5000418458001E0000005E9E9B
:10053000E9FFEEE7ECFFF15CF0FFCEFEF3FFF7CE54
:10054000F7FFDECEFBFF00000000DA630400F0FBE3
:100550000800CCC90D00FBCE1200120D1800A785B3
:100560001D00583A2300C82C29009D5E2F0083D11E
:1005700035002E873C0050814300A6C14A00F04957
:10058000520023000000DCDBE5FF9D11E9FFC9718B
:10059000ECFFC2FDEFFFF0B6F3FFBD9EF7FF9BB689
:1005A000FBFF00000000667C04004F2D09003C1496
:1005B0000E00BA321300578A1800A51C1E003EEB2D
:1005C0002300BDF72900C843300001D1360017A130
:1005D0003D00BAB544009F104C00280000007C1C70
:1005E000E2FF6D3EE5FFC489E8FFD9FFEBFF0DA2F6
:1005F000EFFFBF71F3FF5A70F7FF499FFBFF000049
:100600000000F4930400A05C0900875B0E002A92AE
:10061000130015021900D7AC1E00019424002EB956
:100620002A00F81D310002C43700F1AC3E0071DA37
:1006300045002D0000008362DEFFA570E1FF25A7C5
:10064000E4FF5807E8FF8F92EBFF274AEFFF7E2F6A
:10065000F3FFF943F7FF0089FBFF000000006CAADD
:100660000400B9890900649F0E00ECEC1300D673F6
:100670001900AC351F00FB33250055702B0053ECDF
:1006800031008FA93800A9A93F003200000054B002
:10069000DAFFA6AADDFF52CCE0FF9F16E4FFDB8A5B
:1006A000E7FF592AEBFF6DF6EEFF73F0F2FFCA1970
:1006B000F7FFD673FBFF00000000B5BF040067B46E
:1006C00009008DDF0E009F42140020DF190091B653
:1006D0001F007DCA25006D1C2C00F6AD3200AB80DA
:1006E0003900370000007308D7FFF5EED9FFCBFBC8
:1006F000DCFF3530E0FF778DE3FFDA14E7FFAAC7B0
:10070000EAFF3BA7EEFFE2B4F2FFFAF1F6FFE35F88
:10071000FBFF00000000B9D304007BDC0900B71B1D
:100720000F00E392140077431A00F22E2000D756F0
:100730002600ACBC2C00FC6133003C000000876D3F
:10074000D3FF3A40D6FF3938D9FFC056DCFF069DAB
:10075000DFFF4F0CE3FFDBA5E6FFF76AEAFFEE5C85
:10076000EEFF137DF2FFBBCCF6FF3F4DFBFF000019
:1007700000005FE60400C4010A009A530F0051DD37
:1007800014005CA01A00359E200057D82600425065
:100790002D004100000059E2CFFF3BA1D2FF66844B
:1007A000D5FF078DD8FF54BCDBFF8013DFFFCA9352
:1007B000E2FF713EE6FFB914EAFFEA17EEFF4F4988
:1007C000F2FF3CAAF6FF043CFBFF000000008EF79E
:1007D00004000E240A00E8860F008421150050F55D
:1007E0001A00BE032100454E270046000000D269D2
:1007F000CCFFE514CFFF3AE3D1FFF8D5D4FF49EEA3
:10080000D7FF5B2DDBFF6294DEFF9424E2FF2BDF3A
:10081000E5FF68C5E9FF8DD8EDFFE119F2FFB08A69
:10082000F6FF492CFBFF000000002B0705002843C2
:100830000A0054B50F00145F1500CE411B00F05E96
:1008400021004B0000000307C9FF469ECBFFC6579F
:10085000CEFF9F34D1FFF535D4FFED5CD7FFB1AAB1
:10086000DAFF6E20DEFF55BFE1FF9E88E5FF827D47
:10087000E9FF3D9FEDFF14EFF1FF4A6EF6FF2A1EE0
:10088000FBFF000000001F150500DC5E0A008EDE85
:100890000F009695150053851B00500000001EBDEB
:1008A000C5FF9140C8FF3CE5CAFF32ACCDFF8C9636
:1008B000D0FF6AA5D3FFEAD9D6FF3135DAFF69B890
:1008C000DDFFBE64E1FF613BE5FF843DE9FF626C53
:1008D000EDFF35C9F1FF3D55F6FFBF11FBFF0000ED
:1008E00000004D210500F4760A00480210009FC464
:1008F0001500550000007B8FC2FF1FFFC4FFF38E61
:10090000C7FF0540CAFF6513CDFF270AD0FF642546
:10091000D3FF3766D6FFBFCDD9FF205DDDFF811540
:10092000E1FF0DF8E4FFF205E9FF6140EDFF93A858
:10093000F1FFBF3FF6FF2307FBFF000000009B2BEA
:1009400005003B8B0A002D201000CDCCCC3D0AD7F2
:10095000233C17B7D13877CC2B329595E6241FB1BD
:100960004F0A0000803FCDCCCC3D6F12833A95BF3B
:10097000D6337D1D9026B3CE010C0000204100002F
:10098000C84200401C4620BCBE4CCA1B0E5AAEC515
:100990009D7400000008000201000003040700002D
:1009A00000000000000000000000250028002B00CF
:1009B00000000000240027002A00040404040404AA
:1009C00004040202020202020303030303030102FE
:1009D00004081020408001020408102001020408CD
:1009E0001020DC1F11241FBECFEFD8E0DEBFCDBF2B
:1009F00024E0A8E6B2E001C01D92A737B207E1F7F4
:100A000012E0A0E0B1E0E0EFF6E502C005900D9243
:100A1000A836B107D9F714E0C2EFD4E004C021979B
:100A2000FE010E947529C13FD107C9F70E945F20CE
:100A30000C94762B0C94000091E090931703809314
:100A400039031092180310923A03089508950895F7
:100A500090E0FC01E253F64F24918654964FFC013E
:100A60008491882399F090E0880F991FFC01E0554C
:100A7000F64FA591B491FC01EA55F64F85919491FA
:100A80008FB7F894EC91E22BEC938FBF089590917F
:100A9000EA028091E9022FEF3FEF981748F4E92F1F
:100AA000F0E0EB53FD4F208130E09F5F9093EA022E
:100AB000C90108959091EA028091E9022FEF3FEF7A
:100AC000981748F4E92FF0E0EB53FD4F208130E018
:100AD0009F5F9093EA02C90108950F931F93CF93EC
:100AE000DF93FC01C081D18117861686CE019F70ED
:100AF0009183808390E080E030E020E0DC01AE7FF5
:100B0000AE0FBF1F5C9111964C9180FF1FC025272F
:100B100048E0D901220F331FB7FF02C050E3352749
:100B20004150B9F701968031910541F7D183C083D7
:100B3000232F332722952F7081E06217130609F0C7
:100B400080E0DF91CF911F910F91089510E024274D
:100B50003127DECF90E0FC01EE56F64F2491FC01E8
:100B6000E253F64F3491FC01E654F64FE491EE2344
:100B7000C9F0222339F0233001F1A8F4213019F112
:100B8000223029F1F0E0EE0FFF1FEA55F64FA59154
:100B9000B4918FB7F894EC91611126C030953E2343
:100BA0003C938FBF08952730A9F02830C9F0243036
:100BB00049F7809180008F7D03C0809180008F77FE
:100BC00080938000DFCF84B58F7784BDDBCF84B581
:100BD0008F7DFBCF8091B0008F778093B000D2CF14
:100BE0008091B0008F7DF9CF3E2BDACF3FB7F894DC
:100BF0008091C1029091C202A091C302B091C4023F
:100C000026B5A89B05C02F3F19F00196A11DB11D67
:100C10003FBFBA2FA92F982F8827BC01CD01620FA3
:100C2000711D811D911D42E0660F771F881F991F5E
:100C30004A95D1F708958F929F92AF92BF92CF922B
:100C4000DF92EF92FF926B017C010E94F6054B014F
:100C50005C01C114D104E104F104B9F00E94F6056D
:100C6000681979098A099B09683E734081059105D5
:100C700080F321E0C21AD108E108F10888EE880E5D
:100C800083E0981EA11CB11CE4CFFF90EF90DF9091
:100C9000CF90BF90AF909F908F900895CF93DF93A8
:100CA000EC0189E00E9428058AE00E9428058BE07B
:100CB0000E942805C330D105A1F160F42297E9F024
:100CC00060E089E00E94AA0560E08AE00E94AA052F
:100CD00060E01CC0C430D10551F1259789F761E06F
:100CE00089E00E94AA0561E08AE00E94AA0561E00D
:100CF0008BE0DF91CF910C94AA0560E089E00E941F
:100D0000AA0560E08AE00E94AA0561E08BE00E94EB
:100D1000AA0565E070E080E090E0DF91CF910C944F
:100D20001B0660E089E00E94AA0561E0CECF60E08A
:100D300089E00E94AA0561E0E5CFAF92BF92CF9211
:100D4000DF92EF92FF920F931F93CF93DF936C018B
:100D50007B018B01040F151FEB015E01AE18BF086C
:100D6000C017D10759F06991D601ED91FC9101901E
:100D7000F081E02DC6010995892B79F7C501DF9136
:100D8000CF911F910F91FF90EF90DF90CF90BF9088
:100D9000AF900895FC01448155816081718187E69F
:100DA00094E00C949D06FC01538D448D252F30E07A
:100DB000842F90E0821B930B541710F0CF96089568
:100DC00001970895FC01918D828D981761F0A28D95
:100DD000AE0FBF2FB11D5D968C91928D9F5F9F735B
:100DE000928F90E008958FEF9FEF0895FC01918D11
:100DF000828D981731F0828DE80FF11D858D90E07E
:100E000008958FEF9FEF0895FC01918D228D892F1A
:100E100090E0805C9F4F821B91098F739927089502
:100E20008BE393E00E94040721E0892B09F420E082
:100E3000822F089580E090E0892B29F00E9410070E
:100E400081110C9400000895FC01A48DA80FB92F06
:100E5000B11DA35ABF4F2C91848D90E001968F73E2
:100E60009927848FA689B7892C93A089B1898C9101
:100E7000837080648C93938D848D981306C0028850
:100E8000F389E02D80818F7D80830895EF92FF921A
:100E90000F931F93CF93DF93EC0181E0888F9B8D9D
:100EA0008C8D98131AC0E889F989808185FF15C057
:100EB0009FB7F894EE89FF896083E889F98980817A
:100EC0008370806480839FBF81E090E0DF91CF9149
:100ED0001F910F91FF90EF900895F62E0B8D10E06B
:100EE0000F5F1F4F0F731127E02E8C8D8E110CC0DA
:100EF0000FB607FCFACFE889F989808185FFF5CF25
:100F0000CE010E942407F1CFEB8DEC0FFD2FF11DD8
:100F1000E35AFF4FF0829FB7F8940B8FEA89FB8961
:100F200080818062CFCFCF93DF93EC01888D8823BF
:100F3000B9F0AA89BB89E889F9898C9185FD03C03C
:100F4000808186FD0DC00FB607FCF7CF8C9185FF21
:100F5000F2CF808185FFEDCFCE010E942407E9CF3B
:100F6000DF91CF910895089520919902260F33279C
:100F7000331F21323105ECF420911103FC0190E084
:100F800080E0243069F082E00895A09199022191D7
:100F9000AC0147585D4FA40FB52FB11D2C9301969E
:100FA000861798F380919902680F6093990280E008
:100FB000089581E008951092110381E08093100359
:100FC0001092EB0261E082E10E94AA0561E083E1F8
:100FD0000E94AA05E9EBF0E080818E7F808380810A
:100FE0008D7F808388E48093B80085E48093BC0083
:100FF00008951092EA021092E902109218031092DA
:101000003A030E94DB0786E295E09093E802809322
:10101000E70287E295E09093E6028093E502089567
:10102000CF93DF9391E0909378028823B9F0C09139
:10103000B800D091BA008091BC008A7B8093BC003C
:1010400060E082E10E94AA0560E083E10E94AA05B7
:101050000E94DB07D093BA00C093B800DF91CF9114
:101060000895CF92DF92EF92FF920F931F93CF9349
:10107000DF93D0913A0381E0D13208F09CC0C09157
:1010800039030E94F6056B017C01809111038111E7
:101090006CC082E08093110381E0809310038FEF96
:1010A00080930F0310920E03D0930D03A9E1B3E0D8
:1010B000EDEEF2E080E0D8138DC01092EC0280914A
:1010C000EC02CC0FC82BC093EC028091EB02813074
:1010D00009F084C01092EB020E94F6056B017C01BE
:1010E0008091EC028093BB008091130390911403D4
:1010F000A0911503B0911603892B8A2B8B2BA1F09D
:101100000E94F6050091130310911403209115031A
:10111000309116036C197D098E099F090617170770
:101120002807390708F442C08091BC0083FDD8CF5E
:1011300085EC8093BC000E94F6056B017C018091D8
:101140001103823009F44CC080910F038F3F09F4E2
:1011500069C080910F03803209F466C080910F034B
:10116000803309F463C084E026C08091130390911A
:101170001403A0911503B0911603892B8A2B8B2B96
:1011800009F483CF0E94F605009113031091140314
:1011900020911503309116036C197D098E099F0962
:1011A000061717072807390708F06FCF8091120339
:1011B0000E94100885E01092180310923A031092D2
:1011C0001703DF91CF911F910F91FF90EF90DF9068
:1011D000CF9008959D9191938F5F6DCF85EEA9CFAC
:1011E0008091130390911403A0911503B0911603FD
:1011F000892B8A2B8B2B09F4A2CF0E94F605009134
:1012000013031091140320911503309116036C19E8
:101210007D098E099F09061717072807390708F067
:101220008ECFC4CF80E0C7CF82E0C5CF83E0C3CFED
:101230000895E091EA028091E902E81730F4F0E0C5
:10124000EB53FD4F808190E008958FEF9FEF08955D
:101250008091E9029091EA02891B990B0895CF923F
:10126000DF92EF92FF920F931F93CF93DF937C0156
:10127000CB018A0120911703222389F0EB016B0136
:10128000C40ED51ECC15DD0569F06991D701ED912D
:10129000FC910190F081E02DC7010995F3CF642FF7
:1012A0000E94B407C801DF91CF911F910F91FF9069
:1012B000EF90DF90CF900895CF93DF931F92CDB73B
:1012C000DEB76983209117032223F9F020913A03B6
:1012D000203258F021E030E0FC013383228390E09B
:1012E00080E00F90DF91CF91089580911803E82F4F
:1012F000F0E0E75EFC4F998190838F5F8093180345
:1013000080933A0381E090E0ECCF61E0CE0101965A
:101310000E94B407F7CF0F931F93CF938C01C62F72
:10132000FC0184810E941C05F80163856C2B88ED0B
:1013300093E00E945C09CF911F910F910C943108AA
:1013400090E080E00895CF93DF93EC01888199814C
:10135000DC01ED91FC910190F081E02D09952A814D
:101360003B81820F931F9B838A83DF91CF910895E6
:10137000CF93DF93EC0188819981DC01ED91FC91A1
:101380000280F381E02D09952A813B81820F931F12
:101390009B838A83DF91CF9108958F929F92AF9222
:1013A000BF92CF92DF92EF92FF920F931F93CF9352
:1013B000DF93CDB7DEB766970FB6F894DEBF0FBEEA
:1013C000CDBF6C018E01095E1F4F78018AE0882E27
:1013D000912CA12CB12CCB01BA01A50194010E9442
:1013E000D927942F852F605DF80162938F01A901A1
:1013F000692F782F411551056105710561F7A70126
:101400004E1B5F0BBF01C6010E94B80966960FB65E
:10141000F894DEBF0FBECDBFDF91CF911F910F912A
:10142000FF90EF90DF90CF90BF90AF909F908F9004
:101430000895FC012581222339F0F8E02F02900164
:101440001124820F931F089590E080E00895FB011E
:1014500001900020E9F73197AF01461B570BDC01E3
:10146000ED91FC910280F381E02D0994FB01019044
:101470000020E9F73197AF01461B570B0C94B809D0
:101480001F93CF93DF93E2E8F1E01281112379F00B
:10149000329621816213F9CFEC016CE50E94A30919
:1014A000612FCE01DF91CF911F910C94A30961119F
:1014B000F9CF63E971E0DF91CF911F910C94360A67
:1014C0002F923F924F925F926F927F928F929F9254
:1014D000AF92BF92CF92DF92EF92FF920F931F9342
:1014E000CF93DF93CDB7DEB76C970FB6F894DEBF1E
:1014F0000FBECDBF8C011B01DC0114968C9114979B
:101500008F77863009F492C268F58230A0F1129686
:10151000ED90FC901397CC901196DC90843008F0FD
:1015200056C2A701B601C1010E94B809F10182812A
:1015300093816C960FB6F894DEBF0FBECDBFDF91DE
:10154000CF911F910F91FF90EF90DF90CF90BF90C0
:10155000AF909F908F907F906F905F904F903F9053
:101560002F9008958C3069F160F4883009F459C2E5
:101570008A3009F43FC26AE971E0C1010E94360A6B
:10158000E5C1803209F4ECC18034A9F76BE5C101F3
:101590000E94A309F801008111810115110509F4C8
:1015A000DAC1B101C8010E94600AC8010E94190A8B
:1015B0008C01892B09F4CFC16CE2C1010E94A309FF
:1015C000ECCFF801C080D180E280F380A7019601C2
:1015D000C701B6010E94F4248111CDCF20E030E094
:1015E000A901C701B6010E94F424882379F0A7015C
:1015F0009601C701B6010E945F269B01AC01C7019D
:10160000B6010E94F424882309F4B5CF20E030E02D
:10161000A901C701B6010E94F42487FF08C06DE24A
:10162000C1010E94A309F7FAF094F7F8F09420E8BA
:1016300036E948E15BE4C701B6010E94C02787FD97
:1016400081C074E1A72EB12C00E210E0188E1F8A31
:10165000F501E658F64F2591359145915491C70112
:10166000B6010E94C02787FD13C0F501E65BF64F67
:101670002591359145915491C701B6010E945A2593
:101680006B017C012F89388D200F311F388F2F8BF4
:101690001595079534E0A31AB1088CEFA8168FEFC3
:1016A000B806B1F655245A9420E030E0A901C701EC
:1016B000B6010E94C02718160CF04BC02CEA35EC7E
:1016C00047E257E3C701B6010E94F42418160CF450
:1016D00040C0A52DB4E0AB02C0011124B12CA12C57
:1016E000FC01EE59F64F3F019C012658364F490147
:1016F0003FEF531671F1F301EA0DFB1D2591359172
:1017000045915491C701B6010E94F42487FF13C08C
:10171000F401EA0DFB1D2591359145915491C701C6
:10172000B6010E945A256B017C018F89988D801B20
:10173000910B988F8F8B159507955A9494E0A91A61
:10174000B108D6CF00E210E055E0552E188E1F8A62
:10175000ABCFC701B6010E943D274B015C012B01B5
:101760003C0106E080E492E4AFE0B0E0898F9A8F1C
:10177000AB8FBC8F102F01509AE0491651046104C1
:101780007104C8F0698D7A8D8B8D9C8D2AE030E0D4
:1017900040E050E00E94D927298F3A8F4B8F5C8F11
:1017A000C301B2012AE030E040E050E00E94D927B6
:1017B00029013A01DFCFC501B4010E94F9249B0140
:1017C000AC01C701B6010E945E266B017C01698DE8
:1017D0007A8D8B8D9C8D0E94F9249B01AC01C701F1
:1017E000B6010E945A252B013C010E943D276B0146
:1017F0007C010E94F9249B01AC01C301B2010E944B
:101800005E269B01AC010E945F260E943D27C60E0A
:10181000D71EE81EF91E898D9A8DAB8DBC8DC8161A
:10182000D906EA06FB06D8F09FEF891A990AA90A99
:10183000B90AAF89B88DAB2B39F1BAE08B16910498
:10184000A104B10408F1EF89F88D3196F88FEF8B80
:10185000C12CD12C7601812C912C540183942AE047
:10186000422E512C612C712CC701B601A3019201AB
:101870000E94D927672B682B692B51F4111644F469
:1018800069017A011150F0CFC12CD12C7601E7CF3C
:10189000B501A401C1010E94CD09112371F14E01CE
:1018A000F1E18F0E911C012F54019AE0492E512C29
:1018B000612C712C015068F0C701B601A30192019F
:1018C0000E94D927605DD4016E934D0169017A01B0
:1018D000F1CF812F90E0BC0160957095F501E81B78
:1018E000F90B31978EE2808344275527461B570B0F
:1018F0006A0D7B1DC1010E94B809EF89F88DEF2B9D
:1019000029F165E6C1010E94A3090F89188D17FF0F
:1019100007C06DE2C1010E94A3091195019511094B
:10192000FE0177969F018AE0E82EF12CC801B701ED
:101930000E94C527805D82938B01672BB9F7A901AF
:101940004E1B5F0BBF01C1010E94B809D101129665
:101950008D919C91EECD6DE5C1010E94A309F6CF5A
:101960006BE7C1010E94A309F801008111810115F3
:10197000110559F1D8011696CC9016971796DC9060
:1019800062E2C1010E94A3097601F70161917F0122
:10199000662321F0C1010E94400AF7CF62E2C10133
:1019A0000E94A3096AE3C1010E94A309B101C80111
:1019B0000E94600AC8010E94190A8C01892B29F033
:1019C0006CE2C1010E94A309D2CF6DE7C5CF62E2EC
:1019D000C1010E94A3098601E00EF11EE016F10686
:1019E00039F0F80161918F01C1010E94400AF6CFE0
:1019F00062E2B2CFCD90DD90ED90FC90B701A601F0
:101A0000F7FE0BC06DE2C1010E94A30944275527D0
:101A1000BA014C195D096E097F09C1010E94CD0907
:101A200085CD4D915D916D917C91F7CF8C916FE952
:101A300071E0811102C064EA71E0C1010E94360ABE
:101A400075CDCF92DF92EF92FF920F931F93CF93BA
:101A5000DF93D82FC62F0E94F6056B017C01809181
:101A60001103811165C081E08093110380931003FD
:101A70009FEF90930F0310920E039C0F90930D0312
:101A80008093EC028091EC02DD0FD82BD093EC0216
:101A90008091EB02813009F07FC01092EB020E942E
:101AA000F6056B017C018091EC028093BB00809174
:101AB000130390911403A0911503B0911603892B81
:101AC0008A2B8B2BA1F00E94F60500911303109135
:101AD000140320911503309116036C197D098E09AA
:101AE0009F09061717072807390708F442C0809195
:101AF000BC0083FDD8CF85EC8093BC000E94F60526
:101B00006B017C0180911103813009F447C0809101
:101B10000E038C1710F4C0910E03ADEEB2E0E5ECAD
:101B2000F2E080E08C1751F19D9191938F5FFACF95
:101B30008091130390911403A0911503B0911603A3
:101B4000892B8A2B8B2B09F48ACF0E94F6050091F2
:101B500013031091140320911503309116036C198F
:101B60007D098E099F09061717072807390708F00E
:101B700076CF809112030E941008C0E01092EA0212
:101B8000C093E9028C2FDF91CF911F910F91FF90AD
:101B9000EF90DF90CF90089585EEAECF8091130344
:101BA00090911403A0911503B0911603892B8A2BF1
:101BB0008B2B09F4A7CF0E94F60500911303109117
:101BC000140320911503309116036C197D098E09B9
:101BD0009F09061717072807390708F093CFC9CFC1
:101BE000FF920F931F93CF93DF93C82F8B0186E74C
:101BF0000E941C056C2F88ED93E00E945C090E94F6
:101C00003108EC2FE695E77084E0E89FF00111249D
:101C1000E750FC4F61817281838194810E941B0691
:101C200086E70E941C0560E088ED93E00E945C0955
:101C30000E943108D82F63E086E70E94210D0E94A0
:101C40005A05F82E0E945A05C82F0E945A0530E006
:101C500020E0D130C1F0D11119C04C2F50E070E01C
:101C600060E0762F652F542F44276F29482BF80109
:101C70004083518362837383C901DF91CF911F91A8
:101C80000F91FF90089521E030E0F6CF22E030E0A0
:101C9000F3CFFF920F931F93CF93DF93C82F8B0146
:101CA00086E70E941C056C2F88ED93E00E945C097A
:101CB0000E943108EC2FE695E77084E0E89FF00180
:101CC0001124E251FC4F64A575A586A597A50E9435
:101CD0001B0686E70E941C0560E088ED93E00E94E9
:101CE0005C090E943108D82F63E086E70E94210D2D
:101CF0000E945A05F82E0E945A05C82F0E945A05C4
:101D000030E020E0D130C1F0D11119C04C2F50E0AB
:101D100070E060E0762F652F542F44276F29482B01
:101D2000F8014083518362837383C901DF91CF91AE
:101D30001F910F91FF90089521E030E0F6CF22E04F
:101D400030E0F3CF0F931F93CF93DF93C82F8B0116
:101D50008EE10E941C056C2F88ED93E00E945C09C7
:101D60000E94310861E070E080E090E00E941B0674
:101D700063E08EE10E94210D0E945A05C82F0E9447
:101D80005A05D82F0E945A05C5FD0FC0C2FD10C0CC
:101D900020E03D2F282BF8013183208390E080E064
:101DA000DF91CF911F910F91089583E090E0F8CFDC
:101DB00084E090E0F5CF0F931F93CF938C01C62F53
:101DC0000E948B096C2F6460C8010E948B096C2FE4
:101DD0006B7FC8010E948B0983EC90E00197F1F7BB
:101DE000CF911F910F9108950F931F93CF93DF937E
:101DF0008C01D62FC42F607F642B0E94DB0E80E104
:101E0000D89FB00111246C2BC801DF91CF911F9195
:101E10000F910C94DB0E40E061E087E694E00E94B5
:101E2000F40E8BE39FE10197F1F70895CF93DF93D1
:101E3000CDB7DEB728970FB6F894DEBF0FBECDBF83
:101E400098E0E6E0F1E0DE01119601900D929A959E
:101E5000E1F790916F04981708F48FEF90E0880FE6
:101E6000991F21E030E02C0F3D1F820F931FFC01D2
:101E700060816E5F606840E087E694E028960FB668
:101E8000F894DEBF0FBECDBFDF91CF910C94F40E5E
:101E900041E00E94F40E81E090E00895FC0124816D
:101EA0003581232B39F421E0FB018081882349F01F
:101EB00020E007C0808191810E94662B21E0892B60
:101EC000B9F7822F08952F923F924F925F926F92AF
:101ED0007F928F929F92AF92BF92CF92DF92EF92BA
:101EE000FF920F931F93CF93DF93CDB7DEB7C0540C
:101EF000D1090FB6F894DEBF0FBECDBF9AA789A750
:101F000082E090E00E944E0680E40E941C050E9440
:101F10003108811198C386E70E941C050E94310890
:101F2000811191C31092130410921204809119042C
:101F3000811139C008E612E080EAD82E86E70E94B7
:101F40001C056D2D88ED93E00E945C090E9431080C
:101F5000782E62E086E70E94210D0E945A05C82E65
:101F60000E945A057110FFC2FC2CE12C4701882AFF
:101F7000C401D8018D939D938D01892B09F4F3C27F
:101F8000D394D394BEEADB12D9CF609169026295F3
:101F90006F7088E692E00E946D05882309F4E3C221
:101FA00081E080931904BE016B5F7F4F80E50E9442
:101FB000490E892B09F0D7C2BE016F5F7F4F80E4C5
:101FC0000E94490E892B09F0CEC24D815E816F813E
:101FD0007885411551056105710509F4C4C28980F0
:101FE0009A80AB80BC808BA69CA6ADA6BEA6892895
:101FF0008A288B2809F4B7C28091720290917302EB
:10200000B0E0A0E0BA2FA92F982F88274A015B01E2
:10201000881A990AAA0ABB0A8D8A9E8AAF8AB88E44
:10202000609174027091750290E080E0A5019401C6
:102030000E94532807E10E94462949019A01840120
:102040000053184F2F4F3F4F09871A872B873C8724
:102050006D897E898F89988D9B01AC010E945328E0
:1020600089849A84AB84BC8400ED801607E09006D6
:10207000A104B1040CF0ADC2E3E0AE2EB12CC12C32
:10208000D12CE12CF12C00E010E00E94FB2701E2B2
:102090000E9446292FA738AB49AB5AAB6BAB7CAB40
:1020A0008DAB9EAB89849A84AB84BC84BB0C8808BE
:1020B000982C5401898A9A8AAB8ABC8A29853A85E8
:1020C0004B855C856989762F862F962F205D37405A
:1020D000410951096109710981099109322E432E83
:1020E000542E652E762E872E982E292EADE3AA2EFD
:1020F000B12C00E00E94FB27A32CB42CC52CD62CBD
:10210000E72CF82C092D122D0E94FB2704E00E94D9
:102110004629298F3A8F4B8F5C8F6D8F7E8F8F8FE3
:1021200098A3BDE1AB2EB12CC12CD12CE12CF12C0C
:1021300000E010E0232D342D452D562D672D782DF0
:10214000892D922D0E94FB27A32CB42CC52CD62CB4
:10215000E72CF82C092D122D0E94FB2704E00E9489
:10216000462929A33AA34BA35CA36DA37EA38FA307
:1021700098A789849A84AB84BC8404E280160AEF11
:1021800090060FEFA006B0060CF06EC029853A85C8
:102190004B855C856989762F862F962F24523A4F7E
:1021A0004F4F5F4F6F4F7F4F8F4F9F4F322E432EBA
:1021B000542E652E762E872E982E292E01E1A02EE4
:1021C000B12CC12CD12CE12CF12C00E010E00E94AC
:1021D000FB27A32CB42CC52CD62CE72CF82C092DCE
:1021E000122D0E94FB27A98CBA8CCB8CDC8CED8C39
:1021F000FE8C0F8D18A10E946329298F3A8F4B8F77
:102200005C8F6D8F7E8F8F8F98A389E0A82EB12C65
:10221000C12CD12CE12CF12C00E010E0232D342D29
:10222000452D562D672D782D892D922D0E94FB2747
:10223000A32CB42CC52CD62CE72CF82C092D122D50
:102240000E94FB27A9A0BAA0CBA0DCA0EDA0FEA015
:102250000FA118A50E94632929A33AA34BA35CA34D
:102260006DA37EA38FA398A76091700270917102F5
:1022700090E080E02D893E894F89588D0E94532837
:1022800006E00E94462939014A01B62FA72FF82FF0
:10229000E92FA0906C02B0906D02950140E050E0F3
:1022A00060E070E080E090E001E10E942D2959019A
:1022B0006A017B018C019301A4016B2F7A2F8F2F70
:1022C0009E2F0E946329522E432E4FAB58AF69AF09
:1022D0007AAF8BAF9CAF60916E0270916F0290E00D
:1022E00080E02D893E894F89588D0E94532807E050
:1022F0000E94462939014A01B62FA72FF82FE92F4E
:10230000A0906A02B0906B02950140E050E060E05E
:1023100070E080E090E000E10E942D2959016A01FF
:102320007B018C019301A4016B2F7A2F8F2F9E2F9D
:102330000E94632959016A017B018C0169857A85B4
:102340008B859C850E94FB243B014C012FA538A95D
:1023500049A95AA96BA97CA98DA99EA90E946C279D
:102360009B01AC01C401B3010E945E2620E030E075
:1023700048EC52E40E94CB26698B7D8B382E292EA7
:102380009501A601B701C801A9A0BAA0CBA0DCA005
:10239000EDA0FEA00FA118A50E946C29ABA4BCA4BF
:1023A000CDA4DEA445015601C12CD12C760189862D
:1023B0009A86AB86BC86CD86DE86EF86F88A540187
:1023C000CB84DC84E12CF12C00E010E00E94FB27A0
:1023D00005E10E94462939014A01B62FA72FF82F9F
:1023E000E92F252D342D4FA958AD69AD7AAD8BADB0
:1023F0009CADA98CBA8CCB8CDC8CED8CFE8C0F8DBB
:1024000018A10E946C2959016A017B018C0193017A
:10241000A4016B2F7A2F8F2F9E2F0E946C290FE023
:102420000E9446290E946C2720E030E048EC52E4EC
:102430000E94CB26698F7A8F8B8F9C8F80E40E94BD
:102440001C058091120490911304892B09F0E8C0B7
:1024500065EE88ED93E00E945C090E943108F82E39
:1024600063E080E40E94210D0E945A05082F0E941B
:102470005A05182F0E945A05482FBB24B394FB1409
:1024800009F471C0F1106FC060E0702F612B90E013
:1024900080E00027162F272F382FE0E1F0E0C12C35
:1024A00050E8D52EEE24EA94F12CCBA6DCA6EDA6BE
:1024B000FEA6C12CA0E8DA2EA8E9EA2EF12C412CC8
:1024C000512CB0E86B2E712C5301420180229122D5
:1024D000A222B32289288A288B2861F08BA49CA48D
:1024E000ADA4BEA48C209D20AE20BF2008251925B8
:1024F0002A253B2576946794579447948BA49CA4F3
:10250000ADA4BEA4B694A794979487948BA69CA6DA
:10251000ADA6BEA6F694E794D794C7943197A1F6DA
:10252000C42ED12CF12CE12CC016D106E206F30604
:10253000D1F40E94F92420E030E04AEF52E40E94F6
:102540005A2520E030E040E857E30E945A2520E079
:1025500030E040EC50E40E945E266DAF7EAF8FAF5E
:1025600021969FAF219764E072E089A59AA50E9409
:102570004E0F811110C06AEA71E089A59AA50E94E8
:102580004E0F81116AC06FEA71E089A59AA50E9479
:102590004E0F81116BC069897D89832D922DC05C9E
:1025A000DF4F0FB6F894DEBF0FBECDBFDF91CF91E6
:1025B0001F910F91FF90EF90DF90CF90BF90AF9061
:1025C0009F908F907F906F905F904F903F902F9053
:1025D000089515E0A12EB12CC12CD12CE12CF12CA9
:1025E00000E010E00E94FB2706E20E9446292FA788
:1025F00038AB49AB5AAB6BAB7CAB8DAB9EAB19A286
:102600001AA21BA21CA21DA21EA21FA218A6198EEE
:102610001A8E1B8E1C8E1D8E1E8E1F8E18A224CE0F
:1026200065EF88ED93E00E945C090E943108F82E66
:102630006091140470911504809116049091170410
:102640000E941B060DCF80E00E94160F64EB71E024
:1026500087E694E00E94270A9ECF9DAC998A8EACB3
:102660008D8A3FAC21962FAC219795CF998C998A72
:10267000AA8CAD8A3B8C2C8C8ECF2F923F924F929E
:102680005F926F927F928F929F92AF92BF92CF9202
:10269000DF92EF92FF920F931F93CF93DF93CDB70B
:1026A000DEB7ED970FB6F894DEBF0FBECDBF9EA785
:1026B0008DA781E090E00E944E0686E70E941C05EF
:1026C0000E9431088111DEC28091F703811138C068
:1026D00007EE13E030EA532E86E70E941C05652DB5
:1026E00088ED93E00E945C090E943108382E62E078
:1026F00086E70E94210D0E945A05482E0E945A0525
:1027000021E0321609F46CC2F42CE12CD701A82B7D
:10271000CD01F801819391938F0153945394FEEA74
:102720005F12DACF6091E80362956F7087EE93E0F5
:102730000E946D05882309F453C281E08093F7035A
:102740008091F803880FBE016B5F7F4F80650E9408
:10275000F00D892B09F044C28091F803880FBE0167
:102760006F5F7F4F80640E94F00D892B09F038C2A3
:102770004D815E816F817885411551056105710537
:1027800009F42EC2E980FA800B811C81E9A6FAA621
:102790000BA71CA7EF28E02AE12A09F421C28091A7
:1027A000F1039091F203B0E0A0E0BA2FA92F982F87
:1027B00088278A019B01081B190B2A0B3B0B0D8BE9
:1027C0001E8B2F8B388F6091F3037091F40390E090
:1027D00080E0A90198010E94532807E10E94462940
:1027E000DA01C9018053984FAF4FBF4F89879A874D
:1027F000AB87BC876D897E898F89988D9B01AC01E1
:102800000E945328A984BA84CB84DC8400EDA016EE
:1028100007E0B006C104D1040CF00DC2B3E0AB2E4A
:10282000B12CC12CD12CE12CF12C00E010E00E9445
:10283000FB2701E20E9446292FA738AB49AB5AABD0
:102840006BAB7CAB8DAB9EAB89859A85AB85BC852C
:10285000BB0F880B982FDC01898B9A8BAB8BBC8BC1
:1028600029853A854B855C856989762F862F962F39
:10287000205D3740410951096109710981099109B8
:10288000322E432E542E652E762E872E982E292EEC
:102890008DE3A82E00E0232D342D452D562D672DD8
:1028A000782D892D922D0E94FB27A32CB42CC52CAA
:1028B000D62CE72CF82C092D122D0E94FB2704E0C2
:1028C0000E944629298F3A8F4B8F5C8F6D8F7E8FA8
:1028D0008F8F98A39DE1A92EB12CC12CD12CE12C76
:1028E000F12C00E010E0232D342D452D562D672DC1
:1028F000782D892D922D0E94FB27A32CB42CC52C5A
:10290000D62CE72CF82C092D122D0E94FB2704E071
:102910000E94462929A33AA34BA35CA36DA37EA3DF
:102920008FA398A7A984BA84CB84DC8404E2A01680
:102930000AEFB0060FEFC006D0060CF06EC0298576
:102940003A854B855C856989762F862F962F245290
:102950003A4F4F4F5F4F6F4F7F4F8F4F9F4F322EEA
:10296000432E542E652E762E872E982E292EF1E199
:10297000AF2EB12CC12CD12CE12CF12C00E010E0B9
:102980000E94FB27A32CB42CC52CD62CE72CF82CAA
:10299000092D122D0E94FB27A98CBA8CCB8CDC8CC4
:1029A000ED8CFE8C0F8D18A10E946329298F3A8F20
:1029B0004B8F5C8F6D8F7E8F8F8F98A3A9E0AA2E8F
:1029C000B12CC12CD12CE12CF12C00E010E0232DF6
:1029D000342D452D562D672D782D892D922D0E9451
:1029E000FB27A32CB42CC52CD62CE72CF82C092DB6
:1029F000122D0E94FB27A9A0BAA0CBA0DCA0EDA0BD
:102A0000FEA00FA118A50E94632929A33AA34BA3F6
:102A10005CA36DA37EA38FA398A76091EF03709131
:102A2000F00390E080E02D893E894F89588D0E9407
:102A3000532806E00E94462939014A01B62FA72FE4
:102A4000F82FE92FA090EB03B090EC03950140E044
:102A500050E060E070E080E090E001E10E942D290C
:102A600059016A017B018C019301A4016B2F7A2F1C
:102A70008F2F9E2F0E946329298B3FAB48AF59AF00
:102A80006AAF7BAF8CAF9DAF6091ED037091EE03A9
:102A900090E080E02D893E894F89588D0E9453280F
:102AA00007E00E94462939014A01B62FA72FF82FC7
:102AB000E92FA090E903B090EA03950140E050E0CF
:102AC00060E070E080E090E000E10E942D29590173
:102AD0006A017B018C019301A4016B2F7A2F8F2F48
:102AE0009E2F0E94632979018A011B012C016985AF
:102AF0007A858B859C850E94FB244B015C012FA568
:102B000038A949A95AA96BA97CA98DA99EA90E9497
:102B10006C279B01AC01C501B4010E945E2620E038
:102B200030E048EC52E40E94CB263B014C01970177
:102B3000A801B101C201A9A0BAA0CBA0DCA0EDA060
:102B4000FEA00FA118A50E946C29C9A4DAA4EBA4C9
:102B5000FCA456016701E12CF12C8701A986BA86F5
:102B6000CB86DC86ED86FE860F87188BE12CF12C58
:102B700000E010E00E94FB2705E10E9446291901B0
:102B80002A01B62FA72FF82FE92F29893FA948AD91
:102B900059AD6AAD7BAD8CAD9DADA98CBA8CCB8C9B
:102BA000DC8CED8CFE8C0F8D18A10E946C295901D4
:102BB0006A017B018C019101A2016B2F7A2F8F2F6B
:102BC0009E2F0E946C290FE00E9446290E946C27CC
:102BD00020E030E048EC52E40E94CB265B016C011F
:102BE00064E072E08DA59EA50E944E0F811108C081
:102BF0006FEA71E08DA59EA50E944E0F81114CC019
:102C0000B301C401ED960FB6F894DEBF0FBECDBF81
:102C1000DF91CF911F910F91FF90EF90DF90CF90B8
:102C2000BF90AF909F908F907F906F905F904F90EC
:102C30003F902F900895E5E0AE2EB12CC12CD12C01
:102C4000E12CF12C00E010E00E94FB2706E20E943C
:102C500046292FA738AB49AB5AAB6BAB7CAB8DABDE
:102C60009EAB19A21AA21BA21CA21DA21EA21FA2E9
:102C700018A6198E1A8E1B8E1C8E1D8E1E8E1F8EF0
:102C800018A2CBCE80E00E94160F67EC71E087E6B9
:102C900094E00E94270AB4CF35014601B1CF2F92AC
:102CA0003F924F925F926F927F928F929F92AF92DC
:102CB000BF92CF92DF92EF92FF920F931F93CF9329
:102CC000DF93CDB7DEB760970FB6F894DEBF0FBEC7
:102CD000CDBF98878F8390E080E00E944E0680E40D
:102CE0000E941C050E9431088111F7C01092E50373
:102CF0001092E40380E40E941C0563EF88ED93E0EA
:102D00000E945C090E94310862E370E080E090E07C
:102D10000E941B0663E080E40E94210D0E945A0578
:102D2000082F0E945A05182F0E945A05482F60E06C
:102D3000702F612B90E080E00027162F272F382F6F
:102D4000E0E1F0E0812C50E8952EAA24AA94B12C61
:102D5000C12CA0E8DA2EA8E9EA2EF12CCD86DE8679
:102D6000EF86F88A412C512CB0E86B2E712C730140
:102D70006201C022D122E222F322CD28CE28CF2820
:102D800061F0CD84DE84EF84F888C820D920EA2061
:102D9000FB200C251D252E253F25769467945794FE
:102DA0004794B694A79497948794CD84DE84EF8457
:102DB000F888F694E794D794C794CD86DE86EF869C
:102DC000F88A3197A1F6842E912CB12CA12C801673
:102DD0009106A206B30609F053C00E94F92422E529
:102DE00038EB4FE253E40E945A2520E030E040E8FF
:102DF00057E30E945A2526E636E64BE352E40E944A
:102E00005E2669837A838C879B8780E40E941C05F9
:102E100065EF88ED93E00E945C090E94310862E34F
:102E200070E080E090E00E941B0663E080E40E9476
:102E3000210D0E945A05082F0E945A05182F0E9442
:102E40005A050E94310860E0702F612B90E080E00D
:102E50000E94F92420E030E04AEF52E40E945A2513
:102E600020E030E040E857E30E945A2520E030E0BF
:102E700040EC50E40E945E2669877A87382E292E1E
:102E800064E072E08F8198850E944E0F811108C026
:102E90006AEA71E08F8198850E944E0F811127C0E8
:102EA00069817A818C859B8560960FB6F894DEBF28
:102EB0000FBECDBFDF91CF911F910F91FF90EF908B
:102EC000DF90CF90BF90AF909F908F907F906F904A
:102ED0005F904F903F902F90089580E00E94160FD2
:102EE0006AED71E087E694E00E94270AD9CFD98481
:102EF000D982EA84EA823C862B86D2CFCF92DF92B7
:102F0000EF92FF920F931F93CF93DF93FC01848185
:102F1000982F9F7739F480788062848311821082A1
:102F200013821282848185FD0BC080E090E0DF91E6
:102F3000CF911F910F91FF90EF90DF90CF90089568
:102F40006115710591F3EA017B016F010081118127
:102F50000115110589F1D80116966D917C91C70173
:102F60000E94662B892B31F1C8010E94190A8C013D
:102F7000EFCF3897FD83EC833097B9F2E601AA8151
:102F8000BB81109791F0CF018A1B9B0B23E0959595
:102F900087952A95E1F715968C93FB83EA83158232
:102FA0001482F782E682CF01C2CFF983E883FB83E4
:102FB000EA83F5CFC801BBCFEC81FD818A819B817B
:102FC0000896E817F907A8F681E08887AECF0F9337
:102FD0001F93CF93DF93EC0188819981009759F07B
:102FE0002A813B812617370730F081E0DF91CF91AE
:102FF0001F910F9108958B016F5F7F4F0E94A02A50
:10300000009759F0998388831B830A832C813D8123
:10301000232B59F7FC011082E8CF80E0E7CFEF9235
:10302000FF920F931F93CF93DF936115710541F4C6
:1030300080E0DF91CF911F910F91FF90EF90089565
:1030400041155105B1F07B01EC010C811D81040F8C
:10305000151FB8010E94E717882351F32881398191
:103060008C819D81B701820F931F0E946F2B1D835E
:103070000C8381E0DECFCF93DF93EC0188819981CF
:10308000009711F00E94172A198218821D821C8253
:103090001B821A82DF91CF910895CF93DF93EC01C9
:1030A000FB0101900020E9F73197AF01461B570B58
:1030B0000E940F18811103C0CE010E943B18CE015F
:1030C000DF91CF910895CF93DF93EC01FB01448111
:1030D0005581608171810E940F18811103C0CE015A
:1030E0000E943B18CE01DF91CF910895EF92FF929D
:1030F0000F931F93CF93DF93EC017B018A01BA01F9
:103100000E94E71781110BC0CE010E943B18CE012F
:10311000DF91CF911F910F91FF90EF9008951D8344
:103120000C83B701888199810E946F2BF0CFEF92B9
:10313000FF920F931F93CF93DF93CDB7DEB7A19785
:103140000FB6F894DEBF0FBECDBF7C01CB01BA0134
:10315000F7011182108213821282158214828E016D
:103160000F5F1F4F22E044E00E949F220097C9F0AA
:10317000FC0101900020E9F73197AF01481B590B82
:10318000BC01C7010E947618A1960FB6F894DEBF65
:103190000FBECDBFDF91CF911F910F91FF90EF90A8
:1031A0000895C7010E943B18EFCFFB01DC01119687
:1031B0001C921E9213961C921E92129715961C92A8
:1031C0001E9214978617970749F0608171816115E7
:1031D000710521F0448155810C9476180895FC0105
:1031E000118210821382128215821482FB010190D7
:1031F0000020E9F73197AF01461B570B0C94761866
:10320000FC0180819181009711F00C94172A089598
:103210002F923F924F925F926F927F928F929F92E6
:10322000AF92BF92CF92DF92EF92FF920F931F93D4
:10323000CF93DF93CDB7DEB7CF54D1090FB6F89453
:10324000DEBF0FBECDBF8C0164E072E00E944E0F66
:10325000882309F467C464E072E0CE0180960E947E
:10326000EF18CE0180960E944F162B013C0164E0BE
:1032700072E0CE014A960E94EF18CE014A960E9453
:103280003D139B01AC01C301B2010E945F262B01DB
:103290003C0164E072E0CE0144960E94EF18CE013A
:1032A00044960E94630F9B01AC01C301B2010E94CE
:1032B0005F262B013C0164E072E0CE010E960E9475
:1032C000EF1883E090E00E944E06809132040E9445
:1032D0001C050E94310881110FC48091570481118F
:1032E0002CC057E4A52E54E0B52E10EA809132048C
:1032F0000E941C05612F88ED93E00E945C090E94EA
:103300003108E82E62E0809132040E94210D0E9473
:103310005A05082F0E945A05E110A1C0902E812C59
:103320009401282BC901D5018D939D935D011E5FEA
:10333000103BE1F681E080935704809132040E94B3
:103340001C0568E488ED93E00E945C090E94310846
:103350006AE070E080E090E00E941B0680913204F9
:103360000E941C0560E088ED93E00E945C090E94C9
:10337000310863E0809132040E94210D0E945A05B9
:10338000082F0E945A05182F0E945A05612F70E0DD
:1033900090E080E0982F872F762F6627802B672F6D
:1033A000782F892F99270E94F92420E030E543ECFB
:1033B00057E40E94CB266B017C0107E414E01FA3B5
:1033C0000EA309E414E0812C912C5401D8016D91D5
:1033D0007D918D0190E080E00E94F924EEA1FFA193
:1033E0005291429132912291FFA3EEA30E945A255D
:1033F000A50194010E945F26A70196010E945A250B
:103400004B015C0121E534E020173107F9F620E09B
:1034100030E040E251E40E945A254B015C0160918A
:1034200051047091520490E080E00E94F9242091B0
:1034300033043091340440913504509136040E9495
:103440005A25A50194010E945F2620E030E048EC57
:1034500052E40E94CB266EA3C72ED82EF92E64E02C
:1034600072E0CE010E960E944E0F882329F0AEA086
:10347000ACA6C8AADCAAF8AE2CA538A94CA958ADB0
:10348000C301B2010E945F2668AF79AF8AAF9BAFDC
:103490006E0108E0C00ED11C64E072E0C6010E941B
:1034A000EF1884E090E00E944E068EE10E941C0519
:1034B0000E94310881112CC38091580481113AC0B7
:1034C00069E574E00E94A20E892B09F0B8C26BE591
:1034D00074E081E00E94A20E892B09F0B0C26DE574
:1034E00074E08AE10E94A20E892B09F0A8C26FE560
:1034F00074E08BE10E94A20E892B09F0A0C261E664
:1035000074E08CE10E94A20E892B09F098C263E658
:1035100074E08DE10E94A20E892B09F090C265E64D
:1035200074E08CE20E94A20E892B09F088C281E02F
:10353000809358048EE10E941C056FEA88ED93E0A9
:103540000E945C090E943108F82E64E670E080E079
:1035500090E00E941B0667E08EE10E94210D8E0123
:103560000F5F1F4F0E945A05D8018D938D01CA1617
:10357000DB06C1F7F11063C28981847209F05FC272
:10358000AA80AEA21B810C818D818E80912CB12CE2
:10359000A12CBA2CA92C982C8824A82A8F81882A9F
:1035A00060915D0470915E04072E000C880B990BEE
:1035B0000E94FB242B013C0160915F047091600428
:1035C000072E000C880B990B0E94FB24A30192018B
:1035D0000E945E266B017C01C501B4010E94FB24A0
:1035E00020E030E040E853E30E945A259B01AC0103
:1035F000C701B6010E945A25A30192010E945F26CD
:103600006AA77BA71C012AEB822E21E0922EF401EF
:1036100065917591859194910E94FB249B01AC0169
:103620006AA57BA5C1010E94C02718160CF007C22D
:10363000E2EFF8E065917591859194910E94FB24E9
:103640009B01AC016AA57BA5C1010E94F424181658
:103650000CF4F5C166246394712C562CF401659129
:103660007591859194910E94FB249B01AC016AA500
:103670007BA5C1010E94C027181684F4C401885A92
:103680009F4F2FEF621A720A39E16316710409F035
:103690003DC2A8E16A2E712CB8E15B2E612F70E06B
:1036A00090E080E0982F872F762F6627AEA08A299A
:1036B000602B805891092091650430916604032E97
:1036C000000C440B550B0E945328E8EEAE2EF3E09D
:1036D000BF2EC12CD12CE12CF12C00E010E00E9477
:1036E0008F282EA33FA348A759A75A9406E1509EBE
:1036F0007001112441E050E0442ED701A40FB51F02
:10370000AA0FBB1FAA0FBB1FAE59BE4FFD0165918B
:10371000759185919491AEA0BFA0C8A4D9A46A1553
:103720007B058C059D054CF44F5F5F4F483151057B
:1037300019F747E150E087E1482E86E1869DB00108
:10374000879D700D112481E090E08CAB3B01680EE9
:10375000791E660C771C660C771C83010E591E4F70
:103760003801F801A590B590C590D4900EA11FA185
:1037700028A539A5A016B106C206D30644F40196C1
:103780008831910511F787E190E017E11CAB28E53E
:10379000529EF0011124EE59FE4FA590B590C590B0
:1037A000D490ACA6BDA6CEA6DFA6F401A590B59098
:1037B000C590D490ACAEBDAECEAEDFAE0FEF040D73
:1037C00010E0F801EE0DFF1DEE0FFF1FEE0FFF1FC3
:1037D000EE59FE4FC590D590E590F490C8AAD9AAAD
:1037E000EAAAFBAAFD01A590B590C590D4902496B5
:1037F000ACAEBDAECEAEDFAE24972CA9215030E0EA
:10380000F901E60FF71FEE0FFF1FEE0FFF1FEE5936
:10381000FE4FC590D590E590F490CCAADDAAEEAA13
:10382000FFAAF301A590B590C590D4902896ACAEB0
:10383000BDAECEAEDFAE2897F801EE0FFF1FEE0F44
:10384000FF1FEE59FE4FC590D590E590F490FA0118
:10385000EE0FFF1FEE0FFF1FEE59FE4F45915591E2
:10386000659174912C964CAF5DAF6EAF7FAF2C9786
:10387000F901EE0FFF1FEE0FFF1FEE59FE4F85906F
:103880009590A590B490FC01EE0FFF1FEE0FFF1F67
:10389000EE59FE4F659175918591949160966CAF4C
:1038A0007DAF8EAF9FAF60976EA17FA188A599A5D0
:1038B00008A919A92AA93BA9601B710B820B930BBC
:1038C0000E94FB242B013C0124966CAD7DAD8EAD96
:1038D0009FAD249728A939A94AA95BA9621B730B3C
:1038E000840B950B0E94FB249B01AC01C301B20128
:1038F0000E94CB262B013C012C966CAD7DAD8EAD8C
:103900009FAD2C976C197D098E099F090E94FB249D
:103910009B01AC01C301B2010E945A252B013C015D
:10392000C701B6010E94FB249B01AC01C301B20197
:103930000E945F266B017C016EA17FA188A599A5DD
:103940000CA91DA92EA93FA9601B710B820B930B1B
:103950000E94FB242B013C0128966CAD7DAD8EAD01
:103960009FAD28972CA93DA94EA95FA9621B730B97
:10397000840B950B0E94FB249B01AC01C301B20197
:103980000E94CB262B013C0160966CAD7DAD8EADC7
:103990009FAD6097681979098A099B090E94FB24E9
:1039A0009B01AC01C301B2010E945A252B013C01CD
:1039B000C501B4010E94FB249B01AC01C301B2010B
:1039C0000E945F26A70196010E945E264B015C01C2
:1039D0006CA57DA58EA59FA50E94FB249B01AC0133
:1039E0006AA57BA5C1010E945E262B013C016CAD3E
:1039F0007DAD8EAD9FAD0CA51DA52EA53FA5601B71
:103A0000710B820B930B0E94FB249B01AC01C30141
:103A1000B2010E94CB269B01AC01C501B4010E94FA
:103A20005A25A70196010E945F266CAF21967FAFB1
:103A3000219725968FAF259729969FAF299764E008
:103A400072E0CE0108960E944E0F811114C060E012
:103A500072E0CE0108960E944E0F882361F01CADE3
:103A60001AA72196AFAC2197ABA625962FAC259728
:103A700029963FAC29972AA53BA5A10168AD79AD50
:103A80008AAD9BAD0E945F2620E030E040EA50E422
:103A90000E94CB266B017C01CE0108960E94001982
:103AA000CE010E960E940019CE0144960E94001984
:103AB000CE014A960E940019CE0180960E940019FC
:103AC000C701B601C15BDF4F0FB6F894DEBF0FBE72
:103AD000CDBFDF91CF911F910F91FF90EF90DF90BD
:103AE000CF90BF90AF909F908F907F906F905F909E
:103AF0004F903F902F90089580E00E94160F6DEE3A
:103B000071E087E694E00E94270AB6CC4C01A5CD6F
:103B100080E00E94160F69E072E087E694E00E9460
:103B2000270AA9CF6AEA71E0C8010E944E0F8823D4
:103B300059F16AEA71E0CE0108960E94EF18CE01B1
:103B400008960E944F166B017C016AEA71E0CE0173
:103B500001960E94EF18CE0101960E94630F9B010F
:103B6000AC01C701B6010E945F2620E030E040E0D2
:103B70005FE30E945A256B017C01CE0101960E94F1
:103B80000019CE0108969ACF6FEA71E0C8010E9431
:103B90004E0F882309F494CF6FEA71E0CE010896A6
:103BA0000E94EF18CE0108960E94630F6B017C0102
:103BB0006FEA71E0CE0101960E94EF18CE010196E6
:103BC0000E943D13CCCF85ED8093BC008091130300
:103BD00090911403A0911503B09116030796A11DAF
:103BE000B11D23E0B695A795979587952A95D1F7AE
:103BF0002091BC0024FD03C0109211030895409150
:103C00001303509114036091150370911603452B13
:103C1000462B472B69F30097A105B10541F02AE235
:103C20002A95F1F700C00197A109B109E1CF809170
:103C300012030C9410081F920F920FB60F921124CA
:103C40002F933F938F939F93AF93BF938091BD0228
:103C50009091BE02A091BF02B091C0023091BC020F
:103C600023E0230F2D3758F50196A11DB11D209398
:103C7000BC028093BD029093BE02A093BF02B0939A
:103C8000C0028091C1029091C202A091C302B09182
:103C9000C4020196A11DB11D8093C1029093C2027E
:103CA000A093C302B093C402BF91AF919F918F9133
:103CB0003F912F910F900FBE0F901F90189526E8FF
:103CC000230F0296A11DB11DD2CF1F920F920FB6E6
:103CD0000F9211242F933F934F935F936F937F9392
:103CE0008F939F93AF93BF93EF93FF938BE393E0F7
:103CF0000E942407FF91EF91BF91AF919F918F9107
:103D00007F916F915F914F913F912F910F900FBED7
:103D10000F901F9018951F920F920FB60F921124BB
:103D20002F938F939F93EF93FF93E0914B03F09129
:103D30004C038081E0915103F091520382FD1BC03E
:103D40009081809154038F5F8F7320915503821768
:103D500041F0E0915403F0E0E55CFC4F958F8093D7
:103D60005403FF91EF919F918F912F910F900FBE70
:103D70000F901F9018958081F4CF1F920F920FB66D
:103D80000F9211242F933F934F935F936F937F93E1
:103D90008F939F93AF93BF93EF93FF938091B9005D
:103DA000887F803609F44AC0F0F5883209F4A7C04C
:103DB00018F5803109F49BC0B8F4882309F4F9C0E0
:103DC000883009F494C0FF91EF91BF91AF919F911A
:103DD0008F917F916F915F914F913F912F910F90B4
:103DE0000FBE0F901F901895883109F488C080325B
:103DF00051F780930F0314C0803409F49DC040F440
:103E00008033B9F38833F9F680930F0385ECB0C0A3
:103E1000803509F485C0883509F496C0883499F650
:103E20000E94E31DD0CF883909F48CC038F588375B
:103E300029F050F4883611F0803729F683E080931A
:103E400011031092BB0257C0883809F47BC0803937
:103E500019F0803809F0B7CF8091BB02803208F0AA
:103E600071C0E091BB0281E08E0F8093BB02809114
:103E7000BB00F0E0E556FD4F80833DC0803B39F04C
:103E8000E0F4803A09F479C0883A09F09CCF84E0E4
:103E90008093110310929A0210929902E091E70226
:103EA000F091E80209958091990281110FC081E09B
:103EB000809399021092790209C0803C09F4A6CF40
:103EC000883C09F4A3CF883B09F07DCFE0919A02AA
:103ED00081E08E0F80939A02F0E0E758FD4F8081D9
:103EE0008093BB0090919A028091990229C08091A1
:103EF000EC028093BB0085EC8093BC0064CF909172
:103F00000E0380910D03981758F5E0910E0381E0A0
:103F10008E0F80930E03F0E0E351FD4F8081E9CFD7
:103F2000E0910E0381E08E0F80930E038091BB0021
:103F3000F0E0E351FD4F808390910E0380910D03DB
:103F40009817C8F285E8D8CFE0910E0381E08E0F74
:103F500080930E038091BB00F0E0E351FD4F80831E
:103F60008091100381115CCF81E08093EB0284EAA1
:103F70008093BC001092110326CF85EC8093BC0087
:103F8000109211038091BB02803230F4E091BB02A9
:103F9000F0E0E556FD4F10826091BB0270E0E091C9
:103FA000E502F091E6028BE992E009951092BB02DE
:103FB0000ACF10920F0334CFCF93DF93EBE3F3E0FC
:103FC0001382128288EE93E0A0E0B0E084839583B0
:103FD000A683B78326E531E03183208325EC30E0EA
:103FE0003587248724EC30E03787268720EC30E0C3
:103FF000318B208B21EC30E0338B228B22EC30E0B4
:10400000358B248B26EC30E0378B268B118E128E6D
:10401000138E148EE8EDF3E013821282848395836D
:10402000A683B78388E691E091838083E7E6F4E096
:10403000138212828AE791E09183808387E28483EE
:1040400080E1818782E0828713861092E5031092D7
:10405000E403C6EED3E0198A88E1EEE0F1E0AAEFCE
:10406000B3E001900D928A95E1F788E1E6E2F1E094
:10407000AAE1B4E001900D928A95E1F780EA90E020
:10408000A0E0B0E08EA79FA7A8ABB9AB81E090E01D
:104090009DA78CA71AAA1BAA87E78093320484E104
:1040A000EEE3F1E0A3E3B4E001900D928A95E1F72D
:1040B0001092570410925804DF91CF910895CF9336
:1040C000DF93CDB7DEB7C059D1090FB6F894DEBF84
:1040D0000FBECDBF789484B5826084BD84B5816005
:1040E00084BD85B5826085BD85B5816085BD8091C3
:1040F0006E00816080936E0010928100809181003B
:104100008260809381008091810081608093810032
:10411000809180008160809380008091B1008460F4
:104120008093B1008091B00081608093B000809155
:104130007A00846080937A0080917A008260809314
:104140007A0080917A00816080937A0080917A0071
:10415000806880937A001092C100E0914B03F09147
:104160004C0382E08083E0914703F0914803108282
:10417000E0914903F0914A038FEC8083109253033E
:10418000E0914F03F091500386E08083E0914D036E
:10419000F0914E03808180618083E0914D03F09126
:1041A0004E03808188608083E0914D03F0914E033F
:1041B000808180688083E0914D03F0914E0380817F
:1041C0008F7D808385E090E00E944E060E94F90773
:1041D0000E94F9070E94F9070E94F9070E94F90757
:1041E0000E94F90710926C0480917104823018F0DB
:1041F00098E090936C0480936F0462E370E080E039
:1042000090E00E941B066091720487E694E00E9491
:104210008B0968EE73E080E090E00E941B0660E38B
:1042200087E694E00E94DB0E0BE416E4C8010197D8
:10423000F1F760E387E694E00E94DB0EC801019786
:10424000F1F760E387E694E00E94DB0E83E592E0FD
:104250000197F1F760E287E694E00E94DB0E60913F
:104260006C04606240E087E694E00E94F40E84E013
:1042700080936D0440E06CE087E694E00E94F40EC9
:104280000E940B0F82E080936E0440E066E087E6B8
:1042900094E00E94F40E40E062E087E694E00E9421
:1042A000F40E8BE39FE10197F1F788E080937204AD
:1042B00060E087E694E00E948B096CE172E087E69B
:1042C00094E00E94270A6EE272E087E694E00E9482
:1042D000270A0E940B0F1E018FE0280E311C8E0151
:1042E0000D581F4F3A8229823C822B821E830D83F8
:1042F00018870F8319861E8664E072E0C8010E9449
:10430000EF18C8010E9408192B013C01C8010E9446
:1043100000196FEA71E0C8010E94EF18C8010E94FD
:1043200008196B017C01C8010E9400196AEA71E05A
:10433000C8010E94EF18C8010E9408194B015C01D6
:10434000C8010E9400190E940B0FB301A201C8010D
:104350000E94971861E372E0CE0187589F4F0E9438
:10436000EF18B801CE0187589F4F0E94631865E38C
:1043700072E00E944D18BC01CE0185579F4F0E94EC
:10438000D518CE0187589F4F0E940019C8010E947E
:10439000001980E00E94160FCE0185579F4F0E94A2
:1043A000CA06B501A401C8010E94971868E372E02B
:1043B000CE0187589F4F0E94EF18B801CE01875851
:1043C0009F4F0E9463186CE372E00E944D18BC017D
:1043D000CE018B579F4F0E94D518CE0187589F4F13
:1043E0000E940019C8010E94001981E00E94160F66
:1043F000CE018B579F4F0E94CA0660E177E280E0B2
:1044000090E00E941B06B701A601C8010E94971800
:1044100061E472E0CE0187589F4F0E94EF18B80107
:10442000CE0187589F4F0E94631865E472E00E9496
:104430004D18BC01CE0181589F4F0E94D518CE0166
:1044400087589F4F0E940019C8010E94001981E0FF
:104450000E94160FCE0181589F4F0E94CA06CE01BE
:1044600081589F4F0E940019CE018B579F4F0E9489
:104470000019CE0185579F4F0E940019AE014F5F72
:104480005F4F6AE472E0CE010A960E947E17FC013B
:10449000892B41F0948190789C6094834082518272
:1044A00062827382AE014F5F5F4F66E572E0CE01BC
:1044B0000A960E947E17FC01892B41F09481907826
:1044C0009C60948380829182A282B382AE014F5F0E
:1044D0005F4F6FE572E0CE010A960E947E17FC01E5
:1044E000892B41F0948190789C609483C082D18222
:1044F000E282F3828BE393E0F8019183808313825D
:104500001282B801CE010A960E94600A6EE272E041
:104510008BE393E00E94270A60ED77E080E090E073
:104520000E941B06E0E0F0E0EF2B09F4DBCE0E94D6
:104530001007882309F4D6CE0E940000D3CEEF9254
:104540000F931F93CF93DF93E80134E047FD34E1ED
:10455000042E000C550B57FF03C05195419551098E
:10456000E32E022F242FAE010E94BD22CE01DF9147
:10457000CF911F910F91EF900895A9E0B0E0E3EC87
:10458000F2E20C941E266A01F22EB02E102FFBE3ED
:10459000AF2EA01608F41BE31F5F012F27E0AE012A
:1045A0004F5F5F4F0E941C24BC018981982F997036
:1045B000913009F43FC09BE2E1FC04C09E2D917054
:1045C000E0FC3AC05E2D5071E82FE87083FF46C0D2
:1045D00084E0911101C083E0EF2DE81B8F1508F0F6
:1045E000E0E0D6018E2F20E2552351F1992329F0E6
:1045F000D6019C93C60101966C0196012D5F3F4F39
:10460000E2FE24C08EE4D6018C9391E411969C9333
:10461000119712968C93D9018E2F90E281111BC0B5
:10462000E20FF32FF11D10828EEF9FEF2996ECE041
:104630000C943A269DE2C6CF90E2C4CF2D938150D0
:104640008111FCCFCE0ED11CE0E0D0CF8EE6D6019A
:104650008C9391E6DBCF9D938150E0CF482F44703F
:1046600082FF3DC084E0911101C083E08F1510F4FA
:10467000EF2DE81BD6018E2F20E2552309F1992357
:1046800029F0D6019C93C60101966C0196012D5F1D
:104690003F4FE2FE1BC089E4D6018C938EE4119655
:1046A0008C93119786E412968C93D9018E2F90E209
:1046B000882309F4B5CF9D938150FACF2D93815073
:1046C0008111FCCFCE0ED11CE0E0D9CF89E6D60116
:1046D0008C938EE611968C93119786E6E4CF9B011E
:1046E00077FF02C030E020E0A1E0B0E0911102C00D
:1046F000B0E0A0E0F9013196AE0FBF1F8B2C912CDA
:10470000BB2009F461C05401EFEFAE1ABE0AAA0D36
:10471000BB1DFA161B0619F014F04F2D4A1B511140
:1047200088C0E3FC59C07601A42FB0E2A1114FC0AC
:10473000C40ED11C992309F45BC040E0D601119648
:10474000F60190836D01552309F448C0012F060F2F
:104750009A81582F507184FF03C0913309F401509E
:1047600010160CF047C0093008F008E0EEE2FE2E0B
:104770005B01A01AB10885019194819491082F3FA3
:10478000320729F4D601FC92F60131966F016217C7
:10479000730794F1021713077CF5DB01A21BB30B1F
:1047A000AA24A394B12CAC0EBD1EAA0DBB1D11965C
:1047B0008C9121503109D601119628153905F4F054
:1047C000F60180836D01DBCFB12CA12CA0CFF701C6
:1047D000B1937F01A150AACF9111B0CFD601942FF0
:1047E00050E302C05D9391509111FCCFC40ED11CD7
:1047F00040E0ACCF01E0BACF80E3DBCF62177307B4
:1048000031F4963388F4953311F4552369F0F601A9
:104810008083FD01842F90E2811108C0A40FB11D97
:104820001C9290E080E002CF81E3F1CF9193815020
:10483000F3CF911183CF8ACF283008F027E03327B8
:10484000DA01990F311D87FD9160009661057105B0
:1048500039F432602E5F3D9330E32A95E1F70895F5
:104860009F3F30F080387105610509F03C5F3C5F87
:104870003D93913008F08068911DDF93CF931F9393
:104880000F93FF92EF92192F987F9695E92F9695A7
:104890009695E90FFF27EE53FF4F99273327EE2414
:1048A000FF24A701E70105900894079428F4360F28
:1048B000E71EF81E491F511D660F771F881F991F9D
:1048C0000694A1F70590079428F4E70EF81E491FF7
:1048D000561FC11D770F881F991F661F0694A1F7E9
:1048E0000590079428F4F80E491F561FC71FD11DC5
:1048F000880F991F661F771F0694A1F705900794EC
:1049000020F4490F561FC71FD81F990F661F771F26
:10491000881F0694A9F784911095177041F0D695D9
:10492000C79557954795F794E7941A95C1F7E8E628
:10493000F0E06894159015913591659195910590E9
:104940007FE27395E118F10A430B560BC90BD009AE
:10495000C0F7E10CF11E431F561FC91FD01D7EF486
:10496000703311F48A95E6CFE894015030F0080FC7
:104970000AF40027021708F4202F2395022F7A3318
:1049800028F079E37D932A95E9F710C07D932A9565
:1049900089F6069497956795379517951794E118BA
:1049A000F10A430B560BC90BD00998F023957E9161
:1049B00073957A3308F070E37C932013B8F77E91F7
:1049C00070617D9330F0839571E37D9370E32A9558
:1049D000E1F71124EF90FF900F911F91CF91DF919C
:1049E000992787FD909508950E94362508F481E067
:1049F0000895E89409C097FB3EF4909580957095D2
:104A000061957F4F8F4F9F4F9923A9F0F92F96E91A
:104A1000BB279395F695879577956795B795F1118F
:104A2000F8CFFAF4BB0F11F460FF1BC06F5F7F4F2C
:104A30008F4F9F4F16C0882311F096E911C077233E
:104A400021F09EE8872F762F05C0662371F096E847
:104A5000862F70E060E02AF09A95660F771F881F16
:104A6000DAF7880F9695879597F90895990F0008BA
:104A7000550FAA0BE0E8FEEF16161706E807F90730
:104A8000C0F012161306E407F50798F0621B730BCB
:104A9000840B950B39F40A2661F0232B242B252B4C
:104AA00021F408950A2609F4A140A6958FEF811DEF
:104AB000811D08950E946D250C94DE250E94D0254D
:104AC00038F00E94D72520F0952311F00C94C725CB
:104AD0000C94CD2511240C9412260E94EF2570F31E
:104AE000959FC1F3950F50E0551F629FF001729F93
:104AF000BB27F00DB11D639FAA27F00DB11DAA1FA2
:104B0000649F6627B00DA11D661F829F2227B00DEE
:104B1000A11D621F739FB00DA11D621F839FA00D79
:104B2000611D221F749F3327A00D611D231F849FC9
:104B3000600D211D822F762F6A2F11249F57504020
:104B40009AF0F1F088234AF0EE0FFF1FBB1F661F9B
:104B5000771F881F91505040A9F79E3F510580F064
:104B60000C94C7250C9412265F3FE4F3983ED4F3CF
:104B7000869577956795B795F795E7959F5FC1F708
:104B8000FE2B880F911D9695879597F9089597F9B3
:104B90009F6780E870E060E008959FEF80EC0895E3
:104BA00000240A941616170618060906089500240C
:104BB0000A9412161306140605060895092E039486
:104BC000000C11F4882352F0BB0F40F4BF2B11F4FA
:104BD00060FF04C06F5F7F4F8F4F9F4F089557FD59
:104BE0009058440F551F59F05F3F71F04795880F5B
:104BF00097FB991F61F09F3F79F0879508951216F2
:104C000013061406551FF2CF4695F1DF08C016169D
:104C100017061806991FF1CF86957105610508944E
:104C20000895E894BB2766277727CB0197F9089565
:104C30002F923F924F925F926F927F928F929F92AC
:104C4000AF92BF92CF92DF92EF92FF920F931F939A
:104C5000CF93DF93CDB7DEB7CA1BDB0B0FB6F8944B
:104C6000DEBF0FBECDBF09942A88398848885F848B
:104C70006E847D848C849B84AA84B984C884DF80FC
:104C8000EE80FD800C811B81AA81B981CE0FD11DE0
:104C90000FB6F894DEBF0FBECDBFED010895A29F01
:104CA000B001B39FC001A39F700D811D1124911D00
:104CB000B29F700D811D1124911D08955058BB277E
:104CC000AA270E9476260C94DE250E94D02538F073
:104CD0000E94D72520F039F49F3F19F426F40C9454
:104CE000CD250EF4E095E7FB0C94C725E92F0E9433
:104CF000EF2558F3BA17620773078407950720F06A
:104D000079F4A6F50C9411260EF4E0950B2EBA2F2B
:104D1000A02D0B01B90190010C01CA01A0011124C1
:104D2000FF27591B99F0593F50F4503E68F11A166D
:104D3000F040A22F232F342F4427585FF3CF4695FE
:104D400037952795A795F0405395C9F77EF41F1620
:104D5000BA0B620B730B840BBAF09150A1F0FF0FEA
:104D6000BB1F661F771F881FC2F70EC0BA0F621FD6
:104D7000731F841F48F4879577956795B795F795C6
:104D80009E3F08F0B0CF9395880F08F09927EE0F5B
:104D90009795879508950E94DF260C94DE250E9442
:104DA000D72558F00E94D02540F029F45F3F29F024
:104DB0000C94C72551110C9412260C94CD250E94F9
:104DC000EF2568F39923B1F3552391F3951B550B08
:104DD000BB27AA2762177307840738F09F5F5F4FCE
:104DE000220F331F441FAA1FA9F335D00E2E3AF00D
:104DF000E0E832D091505040E695001CCAF72BD025
:104E0000FE2F29D0660F771F881FBB1F2617370775
:104E10004807AB07B0E809F0BB0B802DBF01FF27A7
:104E200093585F4F3AF09E3F510578F00C94C72598
:104E30000C9412265F3FE4F3983ED4F38695779561
:104E40006795B795F7959F5FC9F7880F911D969560
:104E5000879597F90895E1E0660F771F881FBB1FBC
:104E6000621773078407BA0720F0621B730B840B69
:104E7000BA0BEE1F88F7E09508950E94F72588F099
:104E80009F5798F0B92F9927B751B0F0E1F0660F0E
:104E9000771F881F991F1AF0BA95C9F714C0B1304F
:104EA00091F00E941126B1E008950C941126672F0D
:104EB000782F8827B85F39F0B93FCCF3869577957E
:104EC0006795B395D9F73EF4909580957095619567
:104ED0007F4F8F4F9F4F089597FB16F40E94B02786
:104EE0000C947327E894F92F96EBFF2381F01216A8
:104EF00013061406440B9395F69587957795679559
:104F000057954040FF23B9F71BC099270895882380
:104F100051F49850D2F7872B762F652F542F432FBB
:104F2000322F20E0B1F3121613061406440B882327
:104F30003AF09A95440F551F661F771F881FCAF7CE
:104F400055234AF4440F551F11F460FF04C06F5FEE
:104F50007F4F8F4F9F4F880F9695879597F90895AC
:104F600090958095709560955095409530952195D8
:104F70003F4F4F4F5F4F6F4F7F4F8F4F9F4F089562
:104F80000E94362508F48FEF0895AA1BBB1B51E140
:104F900007C0AA1FBB1FA617B70710F0A61BB70BA9
:104FA000881F991F5A95A9F780959095BC01CD014E
:104FB0000895A1E21A2EAA1BBB1BFD010DC0AA1F5A
:104FC000BB1FEE1FFF1FA217B307E407F50720F072
:104FD000A21BB30BE40BF50B661F771F881F991FED
:104FE0001A9469F760957095809590959B01AC0136
:104FF000BD01CF010895DF93CF931F930F939A9D27
:10500000F02D219FF00D8B9DF00D8A9DE02DF10D6F
:10501000039FF00D029FE00DF11D4E9DE00DF11D6F
:105020005E9DF00D4F9DF00D7F936F93BF92AF92F9
:105030005F934F93D5010E944F268B01AC01D7019E
:105040000E944F26EB01E80FF91FD6010E944A2863
:105050002F913F91D6010E944F26C60FD71FE81F00
:10506000F91FAF91BF910E944A282F913F910E9452
:105070004F26C60FD71FE81FF91FD6010E944F26E3
:10508000E60FF71F9801BE01CF010F911F91CF913D
:10509000DF9108950E944F26460F571FC81FD91F42
:1050A00008F43196089597FB57FF0C9463289F935B
:1050B0008F930E9463286E1B7F0BAF91BF918A0B69
:1050C0009B0B0895E894DF93CF93FC01DB010E94D2
:1050D0004F267F936F93E9019A01AC01BF93AF9381
:1050E0003F932F93DF010E944F2626F46C1B7D0B0C
:1050F000820B930B9E01EB01FC010E944A28AF91A9
:10510000BF912F913F910E944A28BE01CF01F90122
:105110002F913F91CF91DF910895689401C0E89459
:10512000F92FF12B12F00C94C128A0E0B0E0EBE9CC
:10513000F8E20C941E26092E059422F40E941D29E3
:10514000112392F4F0E80F26FFEFE094F09400951D
:105150001095B094C094D094A194BF0ACF0ADF0AEE
:10516000EF0AFF0A0F0B1F0B0E94CC2807FC0E94BE
:105170001D29CDB7DEB7ECE00C943A26689401C047
:10518000E8948F929F92CF93DF930E94CC28DF9177
:10519000CF919F908F90089588249924F401E40181
:1051A000B0E49F93AA279A158B049C04ED05FE0595
:1051B000CF05D007A10798F4AD2FDC2FCF2FFE2FFE
:1051C000E92D982C892E982F872F762F652F542F15
:1051D000432F322F2227B85031F7BF9127C01B2E03
:1051E000BF91BB27220F331F441F551F661F771F18
:1051F000881F991F881C991CEE1FFF1FCC1FDD1FE5
:10520000AA1FBB1F8A149B04EC05FD05CE05DF0514
:10521000A007B10748F08A189B08EC09FD09CE09E0
:10522000DF09A00BB10B21601A94E1F62EF4940172
:10523000AF01BE01CD01000C089560957095809579
:10524000909530954095509521953F4F4F4F5F4F2A
:105250006F4F7F4F8F4F9F4F0895002E083090F073
:10526000982F872F762F652F542F432F322F2227E9
:105270000850F4CF220F331F441F551F661F771F9E
:10528000881F991F0A95B2F7002D089597FD109475
:10529000002E083098F00850232F342F452F562F1A
:1052A000672F782F892F912DF4CF15949795879597
:1052B0007795679557954795379527950A95AAF756
:1052C0001124002D08952A0D3B1D4C1D5D1D6E1DE2
:1052D0007F1D801F911F08952A193B094C095D0904
:1052E0006E097F09800B910B0895EE0FFF1F05904B
:1052F000F491E02D09940F931F93CF93DF938230A5
:10530000910510F482E090E0E0917504F09176044C
:1053100030E020E0B0E0A0E0309799F421153105AD
:1053200009F44AC0281B390B24303105D8F58A818D
:105330009B816115710589F1FB0193838283FE01D5
:1053400011C0408151810281138148175907E0F053
:105350004817590799F4109761F012960C93129719
:1053600013961C933296CF01DF91CF911F910F912D
:1053700008950093750410937604F4CF2115310538
:1053800051F04217530738F0A901DB019A01BD0122
:10539000DF01F801C1CFEF01F9CF9093760480933C
:1053A0007504CDCFFE01E20FF31F8193919322503C
:1053B000310939832883D7CF209173043091740445
:1053C000232B41F4209102013091030130937404A6
:1053D00020937304209100013091010121153105C2
:1053E00041F42DB73EB74091040150910501241BB3
:1053F000350BE0917304F0917404E217F307A0F405
:105400002E1B3F0B2817390778F0AC014E5F5F4F1A
:105410002417350748F04E0F5F1F509374044093D4
:105420007304819391939FCFF0E0E0E09CCFCF9302
:10543000DF930097E9F0FC01329713821282A0916A
:105440007504B0917604ED0130E020E01097A1F4EE
:1054500020813181820F931F209173043091740455
:105460002817390709F061C0F0937404E0937304BE
:10547000DF91CF910895EA01CE17DF07E8F54A8161
:105480005B819E0141155105B1F7E901FB83EA8378
:1054900049915991C40FD51FEC17FD0761F4808124
:1054A00091810296840F951FE901998388838281F7
:1054B00093819B838A83F0E0E0E012968D919C912A
:1054C00013970097B9F52D913C911197CD01029654
:1054D000820F931F209173043091740428173907A9
:1054E00039F6309751F51092760410927504B09306
:1054F0007404A0937304BCCFD383C28340815181D1
:10550000840F951FC817D90761F44E5F5F4F8881DC
:105510009981480F591F518340838A819B819383CE
:1055200082832115310509F0B0CFF0937604E09322
:1055300075049ECFFD01DC01C0CF13821282D7CF4C
:10554000B0E0A0E0E6EAFAE20C941A268C0100979B
:1055500051F4CB010E947B298C01C801CDB7DEB785
:10556000E0E10C943626FC01E60FF71F9C01225067
:105570003109E217F30708F49DC0D901CD91DC9100
:105580001197C617D70798F0C530D10530F3CE0173
:1055900004978617970708F3C61BD70B2297C1936A
:1055A000D1936D937C93CF010E94172AD6CF5B01D4
:1055B000AC1ABD0A4C018C0E9D1EA0917504B091D1
:1055C0007604512C412CF12CE12C109731F580916F
:1055D0007304909174048815990509F05CC046160F
:1055E000570608F058C08091000190910101009782
:1055F00041F48DB79EB74091040150910501841B81
:10560000950BE817F90708F055C0F0937404E09380
:105610007304F90171836083A0CF8D919C911197E0
:1056200012966C90129713967C901397A815B90553
:1056300059F56C0142E0C40ED11CCA14DB0420F100
:10564000AC014A195B09DA011296159780F0628263
:10565000738251834083D9016D937C93E114F104EB
:1056600071F0D7011396FC93EE93129776CF2296A2
:105670008C0F9D1FF90191838083F301EFCFF0938D
:105680007604E093750469CF4816590608F42C0196
:105690007D01D3019ACFCB010E947B297C01009729
:1056A00049F0AE01B8010E945D2BC8010E94172A83
:1056B000870153CF10E000E050CFFB01DC0102C0B6
:1056C00001900D9241505040D8F70895FB01DC0144
:1056D0008D91019080190110D9F3990B0895FB0168
:1056E000DC0101900D920020E1F70895F894FFCFBE
:1056F0000000770480000000400014005400010006
:105700000000020000000300000005000000090086
:105710000000110000000100000002000000030072
:105720000000050000000900000012000000000059
:10573000C0BF0000803F000000C0000080400000AB
:1057400000C00000000046079D06D306930704072B
:10575000E206F606000000005C092F09A0091809FE
:1057600028094705190900000000480F9D06A009F7
:10577000B3072F2F22225C5C6208660C6E0A720D42
:105780007409005C7530303030006E756C6C0074DC
:105790007275650066616C73650068756D6900708F
:1057A000726573004E6170616B612073656E7A6F14
:1057B000726A61203321004E6170616B61207365F4
:1057C0006E7A6F726A61203221004E6170616B6186
:1057D0002073656E7A6F726A61203121004E6170AC
:1057E000616B612073656E7A6F726A61203421008B
:1057F0006F626A5F74656D70004E6170616B6120ED
:1058000073656E7A6F726A61203521005672656D1C
:10581000656E736B6120706F7374616A61000D0A4D
:1058200000543A2000204300483A200020255248E6
:1058300000503A2000206850610074656D706572F8
:1058400061747572650068756D696469747900705A
:08585000726573737572650047
:107E0000112484B714BE81FFF0D085E080938100F7
:107E100082E08093C00088E18093C10086E0809377
:107E2000C20080E18093C4008EE0C9D0259A86E02C
:107E300020E33CEF91E0309385002093840096BBD3
:107E4000B09BFECF1D9AA8958150A9F7CC24DD24C4
:107E500088248394B5E0AB2EA1E19A2EF3E0BF2EE7
:107E6000A2D0813461F49FD0082FAFD0023811F036
:107E7000013811F484E001C083E08DD089C08234E0
:107E800011F484E103C0853419F485E0A6D080C0E4
:107E9000853579F488D0E82EFF2485D0082F10E0AE
:107EA000102F00270E291F29000F111F8ED06801E7
:107EB0006FC0863521F484E090D080E0DECF843638
:107EC00009F040C070D06FD0082F6DD080E0C81688
:107ED00080E7D80618F4F601B7BEE895C0E0D1E017
:107EE00062D089930C17E1F7F0E0CF16F0E7DF06D8
:107EF00018F0F601B7BEE89568D007B600FCFDCFD4
:107F0000A601A0E0B1E02C9130E011968C91119780
:107F100090E0982F8827822B932B1296FA010C0160
:107F200087BEE89511244E5F5F4FF1E0A038BF0790
:107F300051F7F601A7BEE89507B600FCFDCF97BE46
:107F4000E89526C08437B1F42ED02DD0F82E2BD052
:107F50003CD0F601EF2C8F010F5F1F4F84911BD097
:107F6000EA94F801C1F70894C11CD11CFA94CF0C13
:107F7000D11C0EC0853739F428D08EE10CD085E9AC
:107F80000AD08FE07ACF813511F488E018D01DD067
:107F900080E101D065CF982F8091C00085FFFCCF94
:107FA0009093C60008958091C00087FFFCCF809118
:107FB000C00084FD01C0A8958091C6000895E0E648
:107FC000F0E098E1908380830895EDDF803219F02E
:107FD00088E0F5DFFFCF84E1DECF1F93182FE3DFCA
:107FE0001150E9F7F2DF1F91089580E0E8DFEE27F6
:047FF000FF270994CA
:027FFE00040479
:00000001FF
